:100000000C942E040C94A4040C9414080C94A404D2
:100010000C94C4090C94A4040C94A4040C94A4049B
:100020000C94A4040C94A4040C94311E0C94A40409
:100030000C94982C0C94A4040C94A4040C94A40484
:100040000C94A4040C94A4040C94A4040C94A40490
:100050000C94A4040C94ED2C0C94A4040C94A4040F
:100060000C94A4040C94A4040C94A4040C94A40470
:100070000C94A4040C94A4040C94A4040C94A40460
:100080000C94A4040C94A4040C94A4040C94A40450
:100090000C94A4040C94A404450D530D5F0D5F0D46
:1000A000370D5F0D5F0D5F0D5F0D5F0D5F0D5F0D18
:1000B0005F0D5F0D5F0D5F0D5F0D5F0D390D5F0D06
:1000C0003B0D5F0D5F0D5F0D5F0D570D5F0D6E0DED
:1000D000550D5F0D5F0D5F0D5F0D5F0D5F0D5F0DCA
:1000E0005F0D5F0D5F0D5F0D5F0D5F0D2F0D4B0DF4
:1000F0003D0D4F0D5F0D3F0D5F0D430D5F0D4D0D20
:10010000410D510D470D490D5F0D5F0D5F0D5F0DE9
:100110005F0D5F0D5F0D310D330D350D590D5B0D0D
:100120005F0D5F0D5F0D5D0D090E0B0E170E170EA7
:10013000170E170E170E170E0D0E0F0E110E170EAF
:10014000170E0B0E1A0E170E170ED30D090E170EE3
:10015000170E0F0E170E170E170E170E170E170E7F
:10016000110E090EF50D170EF90D170E170E170EBD
:10017000D50D0D0E170E170E030E170E170E170EB8
:10018000D70D150E170EF70D170E0B0E170E170EB7
:10019000070EFB0D170EFD0D0F0E170E170E170E87
:1001A000050EFF0D170E170E170E170E170E170E52
:1001B000170E010E170ED90D170E170E0D0E170E76
:1001C000170E150E170E170E170E170E170E170E09
:1001D000170E170E170EDB0D170E170E170E030E48
:1001E000170E170E170E170E170E170E170E170EE7
:1001F000170E170EDD0D170EDF0DE10D170E170E82
:10020000170EE30DE50DE70D170EE90DEB0D170EBB
:10021000170E170E130EED0D170EF10DEF0DF30D5A
:10022000170E170E170E170E150E5C0EAA0E850E62
:10023000D00EF60EFE0E050F0A0F0E0FA50FA70F1C
:10024000A90FAB0FAD0FB50FB50FB50FAF0FB10FB6
:10025000B30F8910A110B510D010E210ED101111DC
:100260002A11501172114812ED13E615CB157C1CA2
:10027000A31C9B1DA31C9B1DEF1C121D9B1D691D18
:10028000781D85228522BD22BD2238236C2363255B
:10029000632583236325142314231D256325322519
:1002A0005025722530325820005220006973723A6E
:1002B0002530345820007725303258200021435310
:1002C000335F4630210A00214353335F5245414496
:1002D00059210A00214353335F5245534554210AA3
:1002E00000214353325F45305F4630210A002143ED
:1002F00053325F46302120253032580A00214353C3
:10030000325F4530210A00214353325F494E495440
:10031000210A00214353315F45305F253032582197
:100320000A00452575200050257520004D5B783A60
:10033000256420793A256420763A256420683A2598
:100340006420623A253032585D0A000A5B434C5201
:100350005D20004C257520000A4D6F7573653A20AD
:1003600025730A000A4445463A20000A4558503A87
:1003700020000A494E543A20000A4C4F473A2000C8
:100380000A4C4D533A200053257520000A49443A3F
:100390002530345828257325732920000A556E6BA3
:1003A0006E6F776E2049443A205265706F727420E8
:1003B000746F20544D4B20004E4720004F4B2000BF
:1003C0000A353537365F43533832683A005225755F
:1003D00020005725752000572575200057257520CA
:1003E00000582575200041257520004925752000FD
:1003F0005B4348475D20000A2575205052543A253A
:10040000303258204953523A2530345820000A25BA
:1004100075204552523A25303258204953523A25D8
:100420003034582000535B25303258202530325864
:1004300020253032585D2000007B46010203763AC9
:10044000687F6577482B353B6978796439141E3CA1
:100450006A7A1D16041A1F3D6B061B070821203EF1
:100460006C2C19091715223F6D11050B0A1C23402E
:100470006E7E100D182425416F360E0C1227264271
:100480007037380F33132D43717534322F2E447269
:100490007C7D28303174457351504A524D492A545D
:1004A00066594F5C5F4C4B4E62635A5D5E602953E8
:1004B00067585B56576147554842403E3C3A3B457A
:1004C0006843413F3D2B357E697A790078141E7C64
:1004D0006A7B1D16041A1F7F6B061B070821204D1F
:1004E0006C2C19091715224A6D11050B0A1C234C97
:1004F0006E49100D182425516F360E0C1227264F09
:100500007037380F33132D52717534502F2E4E72B1
:10051000397D283065314B735464586776012A77EA
:100520003259745C5F66020362635A5D5E602953F0
:1005300044575B565561474680291E1F20212223C0
:10054000242526272D2E2A2B141A0815171C180CC3
:1005500012132F302878041607090A0B0D0E0F33DB
:10056000343579311D1B06190511103637387D5584
:100570007A2C393A3B3C3D3E3F4041424353475F32
:100580006061565C5D5E57595A5B626346486444DD
:1005900045677B7F650301025250514F68696A6B62
:1005A0006C6D6E6F7071725800494C754A4D734B8B
:1005B0004E767C777E7466540A4C6F6F702073742D
:1005C0006172742E0A000A55534220636F6E666989
:1005D00067757265642E0A000A544D4B3A393665C8
:1005E0003732322F4C5546413A6436613764660AD9
:1005F000003403490042004D002000500043002019
:10060000006B006500790062006F00610072006499
:1006100000200063006F006E0076006500720074B9
:1006200000650072000000080354004D004B0000FC
:10063000000403090409025400030100A032090464
:10064000000001030101000921110100012239000C
:1006500007058103200001090401000103010200D4
:10066000092111010001227F000705820308000112
:100670000904020001030000000921110100012208
:100680002200070583032000011201100100000071
:1006900008EDFEEE1B0102010200010631FF0974A4
:1006A000A1010975150026FF009520750881020932
:1006B00076150026FF00952075089102C0050109F6
:1006C00002A1010901A100850105091901290815E7
:1006D00000250195087501810205010930093115D0
:1006E00081257F95027508810609381581257F953A
:1006F0000175088106050C0A38021581257F9501D0
:1007000075088106C0C005010980A1018502160196
:10071000002637001A81002AB70075109501810064
:10072000C0050C0901A1018503160100269C021ACF
:1007300001002A9C02751095018100C0050109067F
:10074000A101050719E029E71500250195087501A4
:100750008102050819012905950575019102950188
:10076000750391010507190029F71500250195F872
:1007700075018102C0636F6E73756D65723A2025D5
:100780003034580A0073797374656D3A202530341B
:10079000580A000A002530325820006B6579626FD4
:1007A0006172643A20004C45443A20253032580AA0
:1007B0000025583A253031366225730A000A202078
:1007C0003031323334353637383941424344454687
:1007D0000A0064656C5F6B65795F6269743A2063D7
:1007E000616E27742064656C3A20253032580A0007
:1007F0006164645F6B65795F6269743A2063616EFE
:100800002774206164643A20253032580A00290A8E
:10081000002575002F002575005D28002564002047
:1008200000256400200025640020002564007C0071
:1008300025303258006D6F7573656B6579205B628A
:10084000746E7C782079207620685D287265702F20
:1008500061636C293A205B00740B581611241FBE8B
:10086000CFEFD0E2DEBFCDBF04B603FE49C080911A
:10087000210490912204A0912304B0912404873094
:10088000904BA740B04B09F03BC01092210410924E
:100890002204109223041092240414BE0FB6F8947C
:1008A000A89580916000886180936000109260003C
:1008B0000FBE1092010810920008E3E0F0E089E01A
:1008C00080935700E491E695E370E150E33040F403
:1008D000F0E0EE0FFF1FE858FE4F2081318102C08B
:1008E00020E030E280E090E0A2E0B0E0821B930BD9
:1008F000A109B109B595A79597958795FC0109952B
:1009000011E0A0E0B1E0EEE8F2E600E00BBF02C0CB
:1009100007900D92AE37B107D9F724E0AEE7B1E00A
:1009200001C01D92A132B207E1F714E0CEE2D4E09B
:1009300004C02197FE010E942831CC32D107C9F7AB
:100940000E9495190C9445310C940000FF93EF938D
:10095000E0917E01F0917F01309709F00995EF91C8
:10096000FF910895FC018591803011F0EFDFFBCFFE
:100970000895FF27E0E230E247FF0CC0419597FF62
:1009800009C0EDE26095709580959095611D711D8F
:10099000811D911D27FF02C0219530E350E2AA2757
:1009A000660F771F881F991FAA1FA41710F0A41B9A
:1009B00063955A95A9F7AA3008F0A95FA05DAF9397
:1009C000F395611571058105910541F7ED3211F43B
:1009D000EF93F395F21718F43F93F395FBCF8F91B4
:1009E000B5DFFA95E1F70895E991F99185918030A5
:1009F00021F0853219F0AADFF9CF089520E0E894BC
:100A000055915532C1F3503311F4689455915A33CE
:100A100048F4505390F3220F022E220F220F200D84
:100A2000250FF4CF0EF4219589919991533619F33E
:100A3000533729F1533559F1BC0188279927E89498
:100A40005C3621F48991999168945591543639F422
:100A500046EF7EF077FF0DC08FEF9FEF0AC055374E
:100A60004AE039F0583540E121F0523642E009F0D1
:100A70000895FF93EF937DDFEF91FF91B7CFFF9341
:100A8000EF93FC0181918030B9F360DFFBCFFF93DE
:100A9000EF9368DFF1CFDF93CF93CDB7DEB7259625
:100AA000A3DFCF91DF910895FC012AB1938D90953A
:100AB00092239AB99BB1838D892B8BB90895FC0140
:100AC0009AB1838D809589238AB99BB1838D892BB7
:100AD0008BB985E08A95F1F7000099B1838D982351
:100AE00081E009F480E00895FC012BB1948D90958C
:100AF00092239BB99AB1848D892B8AB90895FC0100
:100B00002AB1948D909592239AB99BB1848D892BAB
:100B10008BB90895FC019AB1848D809589238AB997
:100B20009BB1848D892B8BB985E08A95F1F7000004
:100B300099B1848D982381E009F480E008950F93A2
:100B40001F93CF93DF938C01EB01C8010E945F05D7
:100B5000882341F0209731F085E08A95F1F7000075
:100B60002197F3CFCE01DF91CF911F910F9108957F
:100B70000F931F93CF93DF938C01EB01C8010E9469
:100B80005F05811108C0209731F085E08A95F1F763
:100B900000002197F3CFCE01DF91CF911F910F91EC
:100BA0000895CF93DF93EC010E945405CE01DF91AD
:100BB000CF910C947F053BB1FC01238D209523231D
:100BC0002BB93AB1238D232B2AB90C947F05FC0154
:100BD0008CB3938D982B9CBB9DB3838D892B8DBB40
:100BE0000895CF93DF93EC010E94E705CE01DF91DA
:100BF000CF910C94D105FC012DB3938D9095922348
:100C00009DBBCF010C94DB05FC0111821082128286
:100C1000138280E090E8958384831782108608957C
:100C2000CF93DF93EC012E9826982F9827980E9457
:100C3000DB05898D843080F440916900880F22E0C3
:100C400030E0B90102C0660F771F8A95E2F7CB0149
:100C5000842B8093690010C040916A008370880FD4
:100C600022E030E0B90102C0660F771F8A95E2F7F3
:100C7000CB01842B80936A009DB38B8D8095892353
:100C80008DBBCE01DF91CF910C940406CF93DF93FF
:100C9000EC018F8190E001968F709927288530E0D4
:100CA0008217930749F4CE010E940406CE010E94E8
:100CB000E705CE010E94D1052FB7F89498858F8162
:100CC000891751F0FE01E90FF11D81859F5F9F702B
:100CD0009887C82FD0E002C0CFEFDFEF2FBFCF3F04
:100CE0008FEFD80781F08091060480FF0CC0DF935E
:100CF000CF9382EA92E09F938F930E944B050F90CF
:100D00000F900F900F90CE01DF91CF9108950F9328
:100D10001F93CF938C01CAE1C15071F0C8010E94AA
:100D200046068F3F2FEF920749F48FE99FE0019726
:100D3000F1F700C00000F0CF8FEF9FEFCF911F9130
:100D40000F9108952F923F924F925F926F927F92F0
:100D50008F929F92AF92BF92CF92DF92EF92FF92CB
:100D60000F931F93CF93DF93EC01062F1B8280918B
:100D7000060480FF0CC01F926F9386EB92E09F9356
:100D80008F930E944B050F900F900F900F908C81C6
:100D90009D818115904899F08091060480FF19C1CA
:100DA0008C819D819F938F938CEA92E09F938F9388
:100DB0000E944B050F900F900F900F900AC19DB3AA
:100DC0008B8D809589238DBB2BE0A22EBB24B39401
:100DD00010E09924939438E0232E47E0342E56E017
:100DE000452E65E0562E74E0872EE3E07E2EF2E07D
:100DF0006F2EA9EACA2EA2E0DA2ECE010E94DB05F0
:100E00008FE193E00197F1F700C00000CE010E944E
:100E100074058FE193E00197F1F700C00000CE0167
:100E20000E94540568E97AE3CE010E949F05892B50
:100E300011F49B826FC0E12CF12C90E59A95F1F7AB
:100E4000C8010E2C02C0959587950A94E2F780FFA1
:100E500005C0B924CE010E947F0503C0CE010E94C7
:100E6000740562E370E0CE010E94B805892B11F48D
:100E70006B8250C062E370E0CE010E949F05892B17
:100E800011F47B8247C02FEFE21AF20A88E0E816DD
:100E9000F10499F690E59A95F1F7CE01BB2019F08F
:100EA0000E947F0502C00E94740562E370E0CE01DB
:100EB0000E94B805892B11F48B822CC062E370E08C
:100EC000CE010E949F05892B11F45B8223C020E58F
:100ED0002A95F1F7CE010E947F059CE2E92EFF24BE
:100EE000F394CE010E948A05882329F0E114F104CD
:100EF000C9F44B820FC0EF28E1F38CE2E82EFF2407
:100F0000F394CE010E948A05811114C0E114F1040A
:100F1000D1F53B828B81813009F049C0AA94A110A0
:100F20003AC045C085E08A95F1F7000091E0E91AE2
:100F3000F108D7CFEF2869F36CE271E0CE010E948F
:100F4000B805892B11F42B82E5CFCE010E9404064F
:100F5000CE010E94D105CE010E94E705CE01DF91AE
:100F6000CF911F910F91FF90EF90DF90CF90BF90A6
:100F7000AF909F908F907F906F905F904F903F9039
:100F80002F900C94870625E02A95F1F7000081E068
:100F9000E81AF108B6CF1B828091060480FF2DCF9E
:100FA000DF92CF920E944B050F900F9026CF8B813E
:100FB00080618B83CE010E94DB058FE39FE1019767
:100FC000F1F700C00000CE010E94D105CE010E94C1
:100FD000E7058FEF9FEFDF91CF911F910F91FF906A
:100FE000EF90DF90CF90BF90AF909F908F907F90C9
:100FF0006F905F904F903F902F9008951F93CF93E5
:10100000DF93EC01162F6DEE0E94A2068A3F910538
:1010100039F4612FCE01DF91CF911F910C94A2067C
:10102000DF91CF911F9108951F920F920FB60F92EB
:1010300011240BB60F922F933F934F935F938F938F
:101040009F93EF93FF9349B15091B701909107049B
:101050002091A1013091A2012115304819F49093FB
:10106000A3010FC08091A301981B933050F0809191
:10107000A1019091A20190939E0180939D0180E235
:101080001AC12091A1013091A20136952795309384
:10109000A2012093A10181E090E001C0880F5A9540
:1010A000EAF7842349F08091A1019091A201906810
:1010B0009093A2018093A1018091A1019091A2013E
:1010C00099278038910509F450C1A8F48032910520
:1010D00009F44BC138F4009709F447C1409709F46B
:1010E00095C0DEC08034910509F43FC1803591057B
:1010F00009F48CC0D5C0803C910531F148F48039A9
:10110000910509F483C0803A910509F44DC0C8C027
:10111000803D910509F47AC0803E910509F0C0C078
:101120008091A1019091A20190939E0180939D01D5
:101130008091A1019091A201892F99279093A201FA
:101140008093A10183E256C080919F01811123C049
:1011500084E629B19091B801922311F48111EDC078
:1011600029B19091B8019223E1F08111ECC08091F6
:10117000A1019091A20190939E0180939D01809185
:10118000A1019091A201892F99279093A2018093A8
:10119000A10182E22FC080919F01823209F0E5C057
:1011A000E6CF8111E2C0E3CF80919F01811125C07C
:1011B00084E629B19091B801922311F48111C9C03C
:1011C00029B19091B8019223F1F08111C8C08091AA
:1011D000A1019091A20190939E0180939D01809125
:1011E000A1019091A201892F99279093A201809348
:1011F000A10181E280939F016BC080919F018132A8
:1012000009F0B3C0E4CF8111B0C0E1CF8091A1015A
:101210009091A20190939E0180939D018091A101E4
:101220009091A20180399A4A11F482E044C0209141
:10123000A1013091A2018091A1019091A20124E02D
:10124000329F212D33271124217056E096958795E2
:101250005A95E1F78227982F9E7F29F0982F96952F
:1012600081708927F8CF811102C081E024C080916C
:10127000A1019091A20197FF02C080E101C081E12C
:1012800080939F018091A1019091A20126E0969503
:1012900087952A95E1F79093A2018093A10118C048
:1012A00010929F018091A1019091A20190939E01C3
:1012B00080939D0180E88093A0019BB18091B8014B
:1012C000282F209592239BB99AB1892B8AB92EC0D9
:1012D0002091A1013091A2018091A401E82FF0E0BA
:1012E000E356FE4F21878F5F8F708093A40190E0BB
:1012F00001968F7099273091A501432F50E08417F4
:10130000950769F42DB38091B801482F40952423A7
:101310002DBB9BB194239BB99AB1892B8AB980913B
:10132000A401831303C080E48093A00180E090E8CF
:101330009093A2018093A10118C095E09A95F1F7CE
:101340000000815006CF25E02A95F1F7000081507A
:1013500007CF95E09A95F1F7000081502ACF25E05C
:101360002A95F1F7000081502BCFFF91EF919F91CB
:101370008F915F914F913F912F910F900BBE0F90E6
:101380000FBE0F901F9018951F920F920FB60F92DD
:1013900011240BB60F922F933F934F935F938F932C
:1013A0009F93EF93FF9349B150919A019091070455
:1013B00020918401309185012115304819F49093D2
:1013C00086010FC080918601981B933050F0809168
:1013D000840190918501909381018093800180E246
:1013E0001AC120918401309185013695279530935B
:1013F00085012093840181E090E001C0880F5A9517
:10140000EAF7842349F080918401909185019068E6
:10141000909385018093840180918401909185014E
:1014200099278038910509F450C1A8F480329105BC
:1014300009F44BC138F4009709F447C1409709F407
:1014400095C0DEC08034910509F43FC18035910517
:1014500009F48CC0D5C0803C910531F148F4803945
:10146000910509F483C0803A910509F44DC0C8C0C4
:10147000803D910509F47AC0803E910509F0C0C015
:1014800080918401909185019093810180938001E6
:101490008091840190918501892F992790938501EE
:1014A0008093840183E256C080918201811123C020
:1014B00084E629B190919B01922311F48111EDC032
:1014C00029B190919B019223E1F08111ECC08091B0
:1014D0008401909185019093810180938001809196
:1014E000840190918501892F99279093850180939C
:1014F000840182E22FC080918201823209F0E5C02E
:10150000E6CF8111E2C0E3CF80918201811125C035
:1015100084E629B190919B01922311F48111C9C0F5
:1015200029B190919B019223F1F08111C8C0809163
:101530008401909185019093810180938001809135
:10154000840190918501892F99279093850180933B
:10155000840181E2809382016BC08091820181329B
:1015600009F0B3C0E4CF8111B0C0E1CF8091840114
:1015700090918501909381018093800180918401F5
:101580009091850180399A4A11F482E044C02091FB
:10159000840130918501809184019091850124E03E
:1015A000329F212D33271124217056E0969587957F
:1015B0005A95E1F78227982F9E7F29F0982F9695CC
:1015C00081708927F8CF811102C081E024C0809109
:1015D00084019091850197FF02C080E101C081E103
:1015E00080938201809184019091850126E09695F7
:1015F00087952A95E1F7909385018093840118C01F
:1016000010928201809184019091850190938101D3
:101610008093800180E8809383019BB180919B013E
:10162000282F209592239BB99AB1892B8AB92EC075
:10163000209184013091850180918701E82FF0E0AD
:10164000E058FE4F21878F5F8F708093870190E075
:1016500001968F70992730918801432F50E08417AD
:10166000950769F42DB380919B01482F4095242361
:101670002DBB9BB194239BB99AB1892B8AB98091D8
:101680008701831303C080E48093830180E090E8A6
:10169000909385018093840118C095E09A95F1F7A5
:1016A0000000815006CF25E02A95F1F70000815017
:1016B00007CF95E09A95F1F7000081502ACF25E0F9
:1016C0002A95F1F7000081502BCFFF91EF919F9168
:1016D0008F915F914F913F912F910F900BBE0F9083
:1016E0000FBE0F901F901895EDE9F1E01182108266
:1016F0001282138220E030E835832483168291E041
:10170000918F128E82E0838F948FE0E8F1E0118256
:1017100010821282138235832483168293E0918F84
:10172000828F88E0838F84E0848F0895262F30E0B5
:1017300094E0359527959A95E1F72770E62FEF709D
:10174000823069F08330A1F08130E1F4F0E080E193
:10175000289FE00DF11D1124E85CFA4F11C0F0E064
:1017600080E1289FE00DF11D1124E854FB4F08C0D3
:10177000F0E080E1289FE00DF11D1124E85CFB4FB3
:101780008491089580E808950F931F93CF93DF937A
:101790008C01EB0169EEFC01808191810E94A2061F
:1017A000F801808191810E9487068883F8018081F9
:1017B00091810E9487068983F801808191810E942E
:1017C00087068A8399279F938F9389811F928F938E
:1017D00088811F928F9385E294E09F938F930E945C
:1017E0004B058DB79EB708960FB6F8949EBF0FBEF7
:1017F0008DBFDF91CF911F910F910895E6EDF1E03C
:101800001192119281E0E63EF807D1F70895CF9347
:10181000DF93EC011B821A821C821D820E94FE0B48
:1018200088819981DF91CF910C9410061F93CF93FB
:10183000DF93FC0184810E94960B87FD20C0182F46
:101840001F70C82FD0E094E0D595C7959A95E1F721
:10185000612F8C2F0E949F20811111C0CC0FDD1FA2
:10186000CA52DE4F81E090E002C0880F991F1A959E
:10187000E2F728813981822B932B99838883DF912A
:10188000CF911F9108951F93CF93DF93FC01848123
:101890000E94960B87FD22C0182F1F70C82FD0E022
:1018A00094E0D595C7959A95E1F7612F8C2F0E940A
:1018B0009F20882399F0CC0FDD1FCA52DE4F81E0B4
:1018C00090E002C0880F991F1A95E2F780959095D5
:1018D000288139818223932399838883DF91CF9153
:1018E0001F91089588EC91E00E94070C8AEB91E02B
:1018F0000C94070C809106048160809306040C947C
:10190000FE0BE82FF0E0EE0FFF1FEA52FE4F808142
:10191000918108950C94FE0B7770E72FF0E098E02A
:10192000899FE00DF11D112484E0EE0FFF1F8A95C1
:10193000E1F76F70E60FF11DEE0FFF1FE050F84961
:10194000859194910895FC018481823070F08430F7
:1019500061F062FB992790F960FD926061FD9460EF
:10196000692F808191810C94FE070895CF93C82F31
:10197000682F88EC91E00E94A30C6C2F8AEB91E019
:10198000CF910C94A30CCF92DF92EF92FF920F9322
:101990001F93CF93DF936C018B010E94C62C7C01B7
:1019A000F601808191810E944606EC01019631F496
:1019B000C7010E94DE2C8017910790F3CE01DF91C2
:1019C000CF911F910F91FF90EF90DF90CF900895EE
:1019D0000F931F93CF93DF93FC0180819181DC01F2
:1019E00012962C912131F9F08F0162EF0E94A2062C
:1019F0008F3FBFEF9B07D1F08A3F9105D1F464EF91
:101A000071E0C8010E94C30C8F3F2FEF9207A1F035
:101A1000D82FCC2764EF71E0C8010E94C30CDE010F
:101A2000A82BCD010BC08DEF9FEF08C08FEF9FEF6C
:101A300005C08EEF9FEF02C080E090E0DF91CF9174
:101A40001F910F910895CF93862F90E0FC017C9712
:101A5000E834F105A0F5E45BFF4F0C94283185E5EF
:101A60003EC08AE53CC08BE53AC08CE538C08DE5C8
:101A700036C08EE534C08FE532C080E630C081E6E6
:101A80002EC082E62CC083E62AC08FE628C081E7FC
:101A900026C082E724C084E722C085E720C087E70C
:101AA0001EC088E71CC08AE71AC08CE718C08FE701
:101AB00016C080E714C089E712C08BE710C0C62F9C
:101AC0001F926F9383E193E09F938F930E944B0546
:101AD0000F900F900F900F908C2F01C084E5CF9145
:101AE0000895CF93DF93EC0199859230A9F128F402
:101AF000992341F09130C9F045C09330B1F1943051
:101B0000D9F140C0603E21F0613E21F482E02BC05B
:101B100081E029C067FD04C0CE010E94160C33C0CD
:101B20006F77CE010E94430C2EC0663359F118F432
:101B30006A3229F427C06A3A29F1663B19F167FD38
:101B400005C0CE010E94230D682F12C06F77CE0111
:101B50000E94230D682F13C06D3121F06D3991F46F
:101B600084E001C083E089870EC0653459F465E5DF
:101B7000CE010E94160C06C0653C21F465E5CE013D
:101B80000E94430C198680E0DF91CF910895862F43
:101B900090E0FC013397E138F10508F048C0EC56BD
:101BA000FF4F0C94283187E108958FE108958CE56B
:101BB000089580E6089582E6089587E2089583E512
:101BC00008958FE2089589E3089587E308958FE3E8
:101BD000089587E408958FE4089586E508958EE5D5
:101BE00008958FE7089580E0089585E608958EE6CC
:101BF00008958FE6089580E3089588E3089580E4CA
:101C0000089588E4089580E5089587E508958FE5AF
:101C1000089588E1089588E0089580E2089580E1BC
:101C2000089589E108958DE6089588E20895862F44
:101C30008F7708958FE008956B35C9F068F46131AE
:101C4000F1F020F46E30C9F484E50895633169F051
:101C5000643599F48BE508956D3559F050F062368E
:101C600051F06C3751F487E7089581E108958DE5CF
:101C700008958AE608958EE00895862F08958FE0EE
:101C80000895613131F0613411F48CE70895862FA5
:101C9000089583E108951F93CF93DF93EC01162FEE
:101CA000EA858E2F90E08930910508F0BDC0FC01D7
:101CB000EB5EFE4F0C9428318A819B8180599B4AB0
:101CC000029720F4CE010E941C0E182F103E69F0DE
:101CD00030F4133871F0143871F46FE792C0113E8C
:101CE00031F0103F41F481E093C082E091C084E084
:101CF0008FC062E086C01A8617FD02C0612F21C026
:101D00000E94FE0B87E093E069C08A819B81805925
:101D10009B4A029720F4CE010E94410E182F1935DC
:101D200009F482C0103F19F0123119F47DC083E02C
:101D30006FC01A8617FD09C0612FCE010E94C70D22
:101D4000682FCE010E94160C70C00E94FE0B8DEF12
:101D500092E044C08A819B8180599B4A029720F47B
:101D6000CE010E941C0E182F133821F0143821F4D4
:101D70006FE757C062E055C01A8617FD02C0612F99
:101D800025C00E94FE0B1F921F938EEE92E09F9340
:101D90008F930E944B050F900F900F900F9024C0CF
:101DA0008A819B8180599B4A029720F4CE010E9430
:101DB000410E182F1A861231C1F11935B1F117FDF4
:101DC00009C0612FCE010E94C70D682FCE010E946D
:101DD000430C2BC00E94FE0B81EE92E09F938F93E9
:101DE0000E944B050F900F908FEF20C0643121F0BF
:101DF000603FD1F486E00CC085E00AC06737A1F4EB
:101E000060E0CE010E94160C0FC0643169F487E0D7
:101E10008A870BC0603F41F488E0FACF673721F42E
:101E200060E0CE010E94430C1A8680E0DF91CF91E2
:101E30001F9108956C3551F018F4633169F00AC0B0
:101E4000663731F06E3731F486E7089581E50895FD
:101E50008EE70895862F08958DE50895CF93DF933B
:101E6000EC016F3B41F028F486E5860F823070F478
:101E700002C06C3F59F41B8684ED92E09F938F93D0
:101E80000E944B050F900F908FEFB1C08B85813072
:101E900009F445C038F0823009F476C0833009F483
:101EA00091C0A4C08A819B8182399B4A21F4CE01D2
:101EB0000E941A0F682F663809F168F46338D1F070
:101EC00020F4603819F582E077C06438A9F06538ED
:101ED000E9F468E61DC06C38A9F030F4673881F089
:101EE0006B38A1F461E014C06D3871F0603F71F49B
:101EF00081E062C062E00CC06FE70AC068E708C01A
:101F000060E006C069E004C06AE002C067FD04C08A
:101F1000CE010E94160C6AC087EC92E02EC01B8690
:101F20008A819B8182399B4A21F4CE010E941A0F3B
:101F3000682F862F90E0FC01E358F109EB30F105A2
:101F4000A0F4E25EFE4F0C94283162E010C06FE70F
:101F50000EC068E60CC068E70AC060E008C061E037
:101F600006C069E004C06AE002C067FD04C0CE019B
:101F70000E94430C3BC08DEB92E09F938F930E9495
:101F80004B050F900F9032C0653279F030F4663116
:101F900071F06E3199F460E00BC0663221F0603F61
:101FA00069F483E009C06DE503C063E501C061E544
:101FB000CE010E94160C04C08B8718C00E94FE0B35
:101FC0001B8614C06E3169F020F46631B9F761E503
:101FD00009C0653221F0663289F76DE503C063E51B
:101FE00001C060E0CE010E94430CEACF80E0DF91A7
:101FF000CF9108958F929F92AF92BF92CF92DF922E
:10200000EF92FF920F931F93CF93DF9300D000D0F6
:102010001F92CDB7DEB78C01DC01ED91FC9183817D
:10202000882391F1E080F180D3800E94C62CFF923A
:10203000EF921F92DF929F938F938EE094E09F9395
:102040008F930E944B05D801ED91FC9111978381EC
:1020500080750FB6F894DEBF0FBECDBF79F4189629
:102060008C9118978B3019F48CE018968C9383819F
:10207000823021F48DE0D80118968C931382D80118
:10208000ED91FC9111821082D801ED91FC91119794
:102090008281882381F1928115968C91981759F14C
:1020A000E080F180D2800E94C62CFF92EF921F92B6
:1020B000DF929F938F9387EF93E09F938F930E947C
:1020C0004B05F80185810FB6F894DEBF0FBECDBF7A
:1020D0000190F081E02D85FF03C0928194FD8EC5B3
:1020E00084FD89C5D801ED91FC91119782811596E7
:1020F0008C9311821082D8011896EC918E2F90E06B
:102100008E30910508F0B9C5FC01E75DFE4F0C94D7
:1021100028310E94C62C9F938F938BEE93E09F9360
:102120008F930E944B050E94C62CF80197838683EB
:10213000808191810E94F10581E0D80118968C93ED
:102140006BC0F801808191810E9446060196C9F713
:10215000D80116968D919C9117970E94DE2C893B91
:102160009B4008F48AC582E02EC50E94C62C9F932E
:102170008F9386EE93E09F938F930E944B056FEFB2
:10218000D8018D919C910E94A2060F900F900F9004
:102190000F908A3F910511F486E015C583E060C376
:1021A000F801808191810E94FB052E98269A2F9834
:1021B000279A0E94C62CD80117969C938E93169747
:1021C00084E04FC3F801868197810E94DE2C853F11
:1021D000914008F452C585E043C32E9826982F9865
:1021E0002798F801808191810E940406D8018D9181
:1021F0009C910E94F1050E94C62C9F938F9381EEC3
:1022000093E09F938F930E944B050E94C62CF80188
:102210009783868386E080870F900F900F900F90B2
:102220002CC5D8018D919C910E944606019609F417
:1022300024C50E94C62C9F938F938CED93E09F93AF
:102240008F930E944B050E94C62CF80197838683CA
:1022500087E0E1CFD80116968D919C9117970E9447
:10226000DE2C853F914018F089E0F8018087D80185
:102270008D919C910E944606019609F4FEC40E942D
:10228000C62C9F938F9387ED93E09F938F930E942B
:102290004B050E94C62CF8019783868388E0BBCF4C
:1022A000D80116968D919C9117970E94DE2C853F40
:1022B000914018F089E0F8018087D8018D919C91B8
:1022C0000E944606019609F4D8C40E94C62C9F932A
:1022D0008F9382ED93E09F938F930E944B0589E04B
:1022E000F80199CFC8010E94E80CD80113969C937D
:1022F0008E9312970E94C62C9F938F938DEC93E040
:102300009F938F930E944B05F801828193810F90D8
:102310000F900F900F90009711F482E010C08F3F44
:10232000BFEF9B0711F481E044C09C012D5F3F4F3C
:102330002230310590F38F3F910529F484E0D801D4
:1023400014968C9363C09C0125583B4A223031057A
:1023500008F46FC48239BBEA9B0709F46AC49C0184
:1023600020593B4A22303105F8F480EC93E09F93EA
:102370008F930E944B0560EFF801808191810E944C
:10238000A2060F900F908A3F910509F049C462E8B8
:10239000D8018D919C910E94A2068A3F910509F077
:1023A0003FC48CEB93E03EC4803BBFEB9B0721F422
:1023B00083E0F80184832AC088278115FBEA9F0700
:1023C00009F4ABCF81152FEB920791F381159F474D
:1023D00079F38CE993E09F938F930E944B0560EF14
:1023E000D8018D919C910E94A2060F900F908A3F78
:1023F000910509F01EC462E0F801808191810E947C
:10240000A2068A3F910509F014C487CFF801228102
:1024100033812E3FFFEF3F0751F02D3F4FEF340741
:1024200049F02115310549F040E251E008C041E290
:1024300051E005C04BE151E002C047E251E0D80154
:1024400014968C91813049F0823051F0833059F0EC
:10245000843061F08CE391E00BC080E391E008C030
:102460008DE291E005C083E391E002C081E491E058
:102470005F934F939F938F933F932F938CE893E0B9
:102480009F938F930E944B058AE0F80180877DC35C
:102490000E94C62C9F938F9387E893E09F938F931E
:1024A0000E944B050F900F900F900F90D80114963B
:1024B0008C91833031F0843079F0823009F07CC126
:1024C00006C068EFF801808191810E94A2060E94F7
:1024D000231F0E94B60C70C165EFD8018D919C91AD
:1024E0000E94A2066AEEF801808191810E94A206F4
:1024F000BE016F5F7F4FC8010E94C40B80E893E06C
:102500009F938F930E944B0568EED8018D919C910B
:102510000E94A20660E0F801808191810E94A206DB
:1025200066EED8018D919C910E94A20666EEF8019C
:10253000808191810E94A20666EED8018D919C91C6
:102540000E94A206BE016F5F7F4FC8010E94C40BAC
:102550000F900F908981882309F47AC08A8188239B
:1025600009F476C089E793E09F938F930E944B050F
:1025700066EEF801808191810E94A20668EED80182
:102580008D919C910E94A20660E0F801808191816A
:102590000E94A20668EED8018D919C910E94A2062D
:1025A00063E0F801808191810E94A20668EED80163
:1025B0008D919C910E94A20662E0F8018081918138
:1025C0000E94A20668EED8018D919C910E94A206FD
:1025D00061E0F801808191810E94A20666EED80137
:1025E0008D919C910E94A20668EEF80180819181F4
:1025F0000E94A20663E0D8018D919C910E94A206E0
:1026000068EEF801808191810E94A20661E0D80104
:102610008D919C910E94A20668EEF80180819181C3
:102620000E94A20662E0D8018D919C910E94A206B0
:1026300068EEF801808191810E94A20663E0D801D2
:102640008D919C910E94A20689E0F801848781C047
:1026500082E793E09F938F930E944B0563EFD8012D
:102660008D919C910E94A20668ECF8018081918175
:102670000E94A20663EFD8018D919C910E94A20650
:1026800064E6F801808191810E94A20663EFD8017F
:102690008D919C910E94A20660E5F8018081918154
:1026A0000E94A206C8010E94E80C292F30E00F907A
:1026B0000F902330310511F080E001C083E0D80194
:1026C0001C968C938BE693E09F938F930E944B050F
:1026D00063EFF801808191810E94A20668ECD80125
:1026E0008D919C910E94A20663EFF80180819181F7
:1026F0000E94A20668ECD8018D919C910E94A206CE
:1027000063EFF801808191810E94A20660E5D80103
:102710008D919C910E94A206C8010E94E80C292F6D
:1027200030E00F900F902430310511F080E001C0AF
:1027300084E0F801848781110EC084E693E09F93C2
:102740008F930E944B0566EFD8018D919C910E945A
:10275000A2060F900F9064EFF801808191810E9492
:10276000A206BE016F5F7F4FC8010E94C40BD80153
:102770001C968C91893049F0833051F0843059F0A7
:10278000882361F083E291E00BC08FE491E008C000
:1027900087E491E005C088E591E002C081E691E020
:1027A0009F938F9388E593E09F938F930E944B05AF
:1027B0000F900F900F900F908BE0F80180870E9490
:1027C000C62C9F938F9383E593E09F938F930E94F2
:1027D0004B050F900F900F900F90D8018D919C9109
:1027E0000E9446064C01019609F447C2F801848113
:1027F000843069F18114910421F0FFEF8F16910468
:1028000069F40E94FE0B0E9435228BE493E09F93B3
:102810008F930E944B050F900F902FC2823069F06A
:10282000833081F0813009F028C2682DC8010E94F0
:10283000710D8F3F09F021C212C0682DC8010E949E
:102840004B0EF7CF682DC8010E942E0FF2CFF80172
:10285000808191810E9487066C01019629F48CE0A9
:10286000D80118968C9309C2F801808191810E9449
:1028700087067C01019699F3D8011C968C91FE0184
:1028800031965F01853028F4833030F4882321F0BD
:10289000DCC08930A1F0D9C0D8011D969C911D974C
:1028A000987F282D2770922B1D969C9384FE02C042
:1028B000DD24DA9485FEC4C0FF24FA94C1C0F80177
:1028C0003585C401887499278834910509F0A9C019
:1028D000C1FEA7C0F0E38F22992495948794959424
:1028E000879420E3C222DD2454E0D594C7945A95FE
:1028F000E1F7C828D92842E0C416D104E1F183E009
:10290000C816D10409F476C0CA94CD2809F0A6C12E
:10291000E6FC17C0A701487055278E2D8F70E7FE83
:1029200007C0452B11F420E001C020EF822B0AC024
:10293000452B11F420E001C020EF982F922B80E06E
:1029400002C080E090E0E4FE05C03860D8011D962A
:102950003C9303C0377FF8013587D8011D962C9131
:102960001D97E5FE04C020611D962C9379C12F7E32
:10297000F801258775C1E0FE05C03064D8011D96B9
:102980003C9303C03F7BF8013587D8011D968C919D
:102990001D97E1FE04C080681D968C9303C08F775D
:1029A000F8018587D8011D968C911D97E2FE04C021
:1029B00080621D968C9303C08F7DF8018587D801B6
:1029C0001D968C911D97E3FE04C080641D968C9328
:1029D00003C08F7BF8018587D8011D968C911D97C8
:1029E000E4FE04C080681D968C9338C18F77F8018F
:1029F000858734C1C70124E0959587952A95E1F72D
:102A0000E7FE03C0806F90E003C0982F9F7080E0C6
:102A1000387F2E2D2770E32EE22AD8011D96EC92E6
:102A20001FC1387F882D8770382BF801358784FEC9
:102A300002C0DD24DA9485FE4DC0FF24FA944AC01A
:102A4000833049F08430C9F045C0833079F4E12CFB
:102A5000F12CC12CD12CD8018D919C910E9487061C
:102A60008F3FBFEF9B07B1F1982F35C0843009F03D
:102A7000F5C0E12CF12CC12CD12CF8018081918181
:102A80000E948706AC018F3FFFEF9F0719F183FD7E
:102A900002C080E001C080EF942F9F70982BD80176
:102AA0001D962C911D9744FF04C028601D962C9301
:102AB00003C0277FF8012587D8011D962C911D970B
:102AC00045FF04C020611D962C9305C02F7EF801A0
:102AD000258701C090E085E0D5011D928A95E9F730
:102AE000F8018585898380E0F0E8CF16D1044CF4A5
:102AF000960141E8C4164FEFD40624F421E83FEFD5
:102B000001C02FE72A83A0E8EA16F10454F49701E4
:102B1000B1E8EB16BFEFFB0614F421E83FEF219577
:102B200001C021E82B83903811F0919501C09FE7F7
:102B30009C83803809F481E88D83C5010E94781F49
:102B400089811F928F938D81282F082E000C330BC3
:102B50003F938F938C81282F082E000C330B3F93CB
:102B60008F938B81282F082E000C330B3F938F936C
:102B70008A81282F082E000C330B3F938F938CE211
:102B800093E09F938F930E944B050FB6F894DEBF9E
:102B90000FBECDBF72C00E94C62C9F938F9387E259
:102BA00093E09F938F930E944B056EEFD8018D9118
:102BB0009C910E94A2060F900F900F900F908A3A5E
:102BC000910521F489E0F801808757C00E94C62C46
:102BD0009F938F9382E293E09F938F930E944B0584
:102BE000C8010E94070C0E94FE0B0E943522D801EA
:102BF00018961C9211CB828185FF74CAD801189651
:102C00008C918B3009F06ECA80EF93E09F938F9385
:102C10000E944B058CE0F80180870F900F9062CAEC
:102C200088EB93E09F938F930E944B050F900F903A
:102C300074CB60EFF801808191810E94A2068A3FE7
:102C4000910509F06ACB63E0D8018D919C910E94B7
:102C5000A2068A3F910509F060CBAACB80E090E004
:102C600025E0D5011D922A95E9F7F80125852983EC
:102C7000E12CF12CC12CD12C3BCF81E00F900F9097
:102C80000F900F900F90DF91CF911F910F91FF90B8
:102C9000EF90DF90CF90BF90AF909F908F9008956E
:102CA00088EC91E00E94FA0F8AEB91E00C94FA0F05
:102CB000E8ECF1E08DE991E0918380831382128248
:102CC0001482158210861186128613861486158644
:102CD0000E94FE0BEAEBF1E080E891E091838083B3
:102CE0001382128214821582108611861286138630
:102CF000148615860C94FE0B80910A030895CF93D9
:102D0000DF9300D01F92CDB7DEB720911804243096
:102D100021F523E029839B838A8382E08093E90065
:102D20008FEF9091E800815095FD06C095ED9A9542
:102D3000F1F700008111F5CF8091E80085FF0DC00B
:102D400040E050E063E070E0CE0101960E944B1B32
:102D50008091E8008E778093E8000F900F900F909D
:102D6000DF91CF910895CF93DF9300D01F92CDB71D
:102D7000DEB720911804243061F519821A821B8273
:102D800022E029838138910520F0805891099B83A6
:102D90008A8382E08093E9008FEF9091E800815070
:102DA00095FD06C095ED9A95F1F700008111F5CFDC
:102DB0008091E80085FF0DC040E050E063E070E0E6
:102DC000CE0101960E944B1B8091E8008E77809384
:102DD000E8000F900F900F90DF91CF910895209110
:102DE0001804243051F522E02093E9002FEF3091B0
:102DF000E800215035FD06C035ED3A95F1F70000A9
:102E00002111F5CF2091E80025FF17C02091100176
:102E1000222341F021E02093F10040E050E065E002
:102E200070E004C040E050E063E070E00E944B1BA3
:102E30008091E8008E778093E8000895CF93DF9328
:102E400020911804243009F04AC0EC01809111014E
:102E50008823E1F0809112018823C1F081E0809302
:102E6000E90081E8815049F09091E80095FD05C0A6
:102E70009AE29A95F1F700C0F5CF8091E80085FFBE
:102E80002EC040E050E060E270E019C081E0809325
:102E9000E90081E8815059F09091E80095FD07C064
:102EA000EFE3F1E03197F1F700C00000F3CF80913C
:102EB000E80085FF14C040E050E068E070E0CE011B
:102EC0000E944B1B8091E8008E778093E80080E29F
:102ED000FE01AAEEB2E001900D928A95E1F7DF9132
:102EE000CF910895CF93C091E801C1110BC00E940A
:102EF000D22C643C79408105910520F081E08093DB
:102F0000E801C1E08C2FCF910895FF920F931F939A
:102F1000CF93DF93D82F0FB607FE83C0809118049C
:102F2000843081F08091030190E0019620910501A9
:102F300030E0822393232091040130E0821793072D
:102F400009F0CBC00E947217811110C0809103015B
:102F500090E001962091050130E082239323209197
:102F6000040130E08217930709F0B7C00E94C62C15
:102F70008C01C091E900CF709091EC00892F817095
:102F800090FD80E8C82B83E08093E90085E0F82E6F
:102F90008091EB0085FD42C08091EB0080FF3EC038
:102FA0008091EE0087FF3AC0809104019091030167
:102FB000981709F457C09091E80095FF8CC0E091F4
:102FC0000101F0910201E80FF11D20818F5F9091C6
:102FD00005018923809304012093F1008091E8008A
:102FE00085FDE2CF8091E80080FFDECF8091E80090
:102FF0008E778093E800F0920001D6CF8091030194
:1030000090E001962091050130E0822393232091E6
:10301000040130E08217930709F44AC0CF70C093CF
:10302000E90040910301842F90E001962091050171
:1030300030E0822393232091040130E0821793072C
:1030400009F44EC0E0910101F0910201E40FF11D7D
:10305000D083809103018F5F909105018923809334
:1030600003013EC08091E80085FF35C0D093F10098
:1030700081E02091F2003091F300232B91F09091A8
:10308000E80090FF0EC09091E80095FF03C01092F9
:10309000F100F9CF9091E8009E779093E800F092CC
:1030A0000001882309F4AACFCF70C093E90018C0AB
:1030B00080910001882309F4B1CF0E94C62C9C01A5
:1030C0008017910711F4890163CF9091000191500D
:1030D00090930001F8CF80E0CCCF40910301B2CFB4
:1030E00080E0DF91CF911F910F91FF900895809123
:1030F0001704811104C00E94B31D0C94151E08957D
:10310000109217040895089542E261EC81E00E9454
:10311000C41A42E061EC82E00E94C41A42E261EC0F
:1031200083E00C94C41A80911A04833009F453C0CC
:1031300030F4813071F0823009F4BAC008958A30D9
:1031400009F4A6C08B3009F478C0893009F0C8C0F2
:1031500020C080911904813A09F0C2C08091E80032
:10316000877F8093E80080911D0490911E04892B35
:1031700021F460E28AEE92E003C060E080E090E03B
:1031800070E00E94981B8091E8008B778093E800A4
:10319000089580911904813209F0A2C080911D0424
:1031A00090911E04892B09F09BC08091E800877FD5
:1031B0008093E8008091E80082FD05C080911804AA
:1031C0008111F8CF8DC08091F10080930A03809126
:1031D000E8008B7781C080911904813A09F080C0A2
:1031E00080911D0490911E04892BA1F48091E80028
:1031F000877F8093E8008091E80080FFFCCF80917A
:1032000011018093F1008091E8008E778093E800AF
:103210000E94F91A80911D0490911E04019709F0F3
:103220005FC08091E800877F8093E8008091E8008C
:1032300080FFFCCF809110014AC080911904813237
:1032400009F04EC080911D0490911E04892B69F4F1
:103250008091E800877F8093E8000E94F91A8091AE
:103260001B04809311010E94352280911D049091CE
:103270001E040197A9F58091E800877F8093E800FC
:103280000E94F91A80911B04809310010C9435223E
:1032900080911904813221F58091E800877F809325
:1032A000E8000E94F91A80911C0480930B03089592
:1032B00080911904813AA1F48091E800877F80937E
:1032C000E8008091E80080FFFCCF80910B038093A1
:1032D000F1008091E8008E778093E8000C94F91A51
:1032E000089580910A038093E90110920A030E94D5
:1032F0008A0C0C9435220C9471190E94722C8091C6
:103300001604882329F00E947F2C81110C94AE1A98
:1033100008950E94942C8091E90180930A030895F6
:103320000C94891908950C949219CF9384B7877FD0
:1033300084BF0FB6F894A89580916000886180934F
:103340006000109260000FBE90E080E80FB6F89425
:1033500080936100909361000FBE85E897E10E9421
:10336000312C86E091E00E941E1F88ED95E00E94BE
:10337000B2040E94720C0E94DD1F0E94B31D0E94C5
:10338000151E78940E94DF1F80911804843029F064
:103390000E94031F0E949219F7CF86EC95E00E94CD
:1033A000B2040E94931988EB95E00E94B204C3E036
:1033B00080911804853019F40E947D19F9CF0E947C
:1033C0005B2C0E94E31F2091E4003091E500809186
:1033D000E6019091E7012817390709F466C080914A
:1033E000E4009091E5009093E7018093E6010E944C
:1033F0007217882309F459C080911804843009F0A9
:1034000054C08091E9008F702091EC00922F917050
:1034100020FD90E8892BC093E9009091EB0090FF8C
:1034200041C09091EE0097FF3DC090910401209122
:103430000301291709F12091E80025FF1DC0E09143
:103440000101F0910201E90FF11D30819F5F209190
:1034500005019223909304013093F1009091E800CC
:1034600095FDE3CF9091E80090FFDFCF9091E800C9
:103470009E779093E800D9CF2091F2003091F3002D
:10348000232B81F09091E80090FF0CC09091E80010
:1034900095FF03C01092F100F9CF9091E8009E775C
:1034A0009093E8008F708093E9000E94031F80CF03
:1034B000292F332723303105C9F060F4213031053D
:1034C00081F02230310509F041C084E590E025E328
:1034D00036E040C021323105E1F02232310531F1D0
:1034E00035C082E190E029E836E034C09927813088
:1034F000910549F028F0029749F5E1EFF5E005C0A4
:10350000E1E3F6E002C0E7E2F6E0849190E09F019B
:1035100021C063307105D0F4660F771FFB01EE58B0
:10352000FE4F2081318189E090E014C06330710545
:1035300068F4FB01EE0FFF1FE459FE4F208131813B
:10354000FB01E759FE4F808190E004C080E090E0ED
:1035500020E030E0FA0131832083089584E189BDC1
:1035600086E189BD09B400FEFDCF8091D8008F7D32
:103570008093D8008091E00082608093E000809189
:10358000E00081FDFCCF0895982F973068F5909367
:10359000E900981739F07091EC002091ED005091FE
:1035A000F00003C0242F762F50E021FD02C09F5F62
:1035B000ECCF3091EB003E7F3093EB003091ED008B
:1035C0003D7F3093ED003091EB0031603093EB00A4
:1035D0007093EC002093ED005093F0002091EE00EA
:1035E00027FDE5CF80E008958F708093E90081E0AA
:1035F00008958091190487FF11C08091E80082FD31
:1036000005C0809118048111F8CF11C08091E800A5
:103610008B770BC080911804882349F08091E800D3
:1036200080FFF8CF8091E8008E778093E8000895BE
:103630002091E4003091E50095E64091EC00842F64
:10364000817040FF23C08091E80080FD1DC0809103
:103650001804882399F0853099F08091EB0085FD5E
:1036600011C04091E4005091E5002417350729F37B
:10367000915011F09A01E1CF84E0089582E008951D
:1036800083E0089581E0089580E008954091E80086
:1036900042FFDDCF0895CF92DF92EF92FF920F931A
:1036A0001F93CF93DF93EC018B017A010E94181BCB
:1036B000811135C0E114F10439F0F7018081918165
:1036C000081B190BC80FD91FC12CD12C01151105CE
:1036D00029F18091E80085FD18C08091E8008E777F
:1036E0008093E8000E94031FE114F10449F0F70100
:1036F00080819181C80ED91ED182C08285E00FC021
:103700000E94181B882311F30AC089918093F1004D
:1037100001501109FFEFCF1ADF0AD8CF80E0DF9107
:10372000CF911F910F91FF90EF90DF90CF90089570
:1037300020911F04309120042617370748F06115A7
:10374000710539F42091E8002E772093E80001C03C
:10375000B901FC0120E06115710569F1809118043F
:103760008823E1F18530E1F18091E80083FD3AC0E2
:103770008091E80082FD2CC08091E80080FFEBCFB3
:103780008091F2009091F3006115710551F088303D
:10379000910538F421912093F1006150710901964F
:1037A000F3CF21E0089709F020E08091E8008E77C0
:1037B0008093E800D0CF2111D1CF0AC080911804A6
:1037C000882361F0853061F08091E80083FD0AC0B4
:1037D0008091E80082FFF2CF80E0089582E00895B2
:1037E00083E0089581E0089520911F043091200422
:1037F0002617370748F06115710539F42091E80064
:103800002E772093E80001C0B901FC0120E061158A
:10381000710581F180911804882309F43EC0853038
:1038200009F43DC08091E80083FD3BC08091E80031
:1038300082FD2DC08091E80080FFE9CF8091F200E9
:103840009091F3006115710559F08830910540F4AD
:1038500024912093F1003196615071090196F2CFC5
:1038600021E0089709F020E08091E8008E778093AE
:10387000E800CDCF2111CECF0AC080911804882353
:1038800061F0853061F08091E80083FD0AC080918D
:10389000E80082FFF2CF80E0089582E0089583E09F
:1038A000089581E008951F93CF93DF93CDB7DEB7DE
:1038B000AA970FB6F894DEBF0FBECDBFE9E1F4E0E2
:1038C0008091F100819324E0E132F207C9F70E9470
:1038D00093188091E80083FF2EC180911904909184
:1038E0001A04492F50E04A30510508F024C1FA016A
:1038F000E95CFE4F0C942831803821F0823809F0C1
:103900001AC108C08091150490911604992389F07A
:1039100082600FC080911D048F70873008F00BC14A
:103920008093E9008091EB0085FB882780F9109255
:10393000E9009091E800977F9093E8008093F10070
:103940001092F100D1C0282F2D7F09F0F4C08823F8
:1039500019F0823061F0EFC080911B04813009F0D2
:10396000EAC0933009F080E0809316042EC0809165
:103970001B0481112AC080911D048F702FEF280F26
:10398000263008F0D8C08093E9002091EB0020FF9A
:103990001CC0933021F48091EB00806214C09091A0
:1039A000EB0090619093EB0021E030E0A90102C0B0
:1039B000440F551F8A95E2F74093EA001092EA00FF
:1039C0008091EB0088608093EB001092E900809179
:1039D000E800877F8093E8000E94F91AACC081114B
:1039E000AAC010911B041F778091E3008078812B7F
:1039F0008093E3008091E800877F8093E8000E9435
:103A0000F91A8091E80080FFFCCF8091E300806884
:103A10008093E300111102C082E001C083E0809333
:103A2000180489C08058823008F085C080911B043A
:103A300090911C048C3D53E0950779F583E08A83CF
:103A40008AE289834FB7F894DE01139620E03EE0C6
:103A500051E2E32FF0E050935700E49120FF03C0C0
:103A6000E295EF703F5FEF708E2F90E0EA3010F03C
:103A7000C79601C0C0968D939D932F5F243149F75F
:103A80004FBF8091E800877F8093E8006AE270E092
:103A9000CE0101960E94981B16C060911D04709182
:103AA0001E04AE014F5F5F4F0E94581ABC01892B64
:103AB00009F441C09091E800977F9093E8008981D4
:103AC0009A810E94F41B8091E8008B778093E80034
:103AD00032C0803881F58091E800877F8093E800CC
:103AE000809114048093F1008091E8008E7772CF6A
:103AF000811121C080911B0490911C049927029789
:103B0000D4F48091E800877F8093E80080911B04C3
:103B1000809314040E94F91A80911404811106C044
:103B20008091E30087FD02C081E001C084E08093C2
:103B300018040E9484188091E80083FF0AC08091D5
:103B4000E800877F8093E8008091EB00806280939B
:103B5000EB00AA960FB6F894DEBF0FBECDBFDF9183
:103B6000CF911F9108950E94241E0E942C1EE0EE0A
:103B7000F0E0808181608083E8EDF0E080818F77E4
:103B8000808319BCA7EDB0E08C918E7F8C938081EF
:103B90008F7E80831092170408950F931F93CF9305
:103BA000DF930E94241E0E942C1EC8EDD0E0888165
:103BB0008F77888388818068888388818F7D8883D8
:103BC000E7EDF0E080818068808319BC10921804D2
:103BD00010921404109216041092150400EE10E0D6
:103BE000F80180818B7F808388818160888342E0B7
:103BF00060E080E00E94C41AE1EEF0E080818E7FF8
:103C00008083E2EEF0E08081816080838081886043
:103C10008083F80180818E7F8083888180618883A2
:103C2000DF91CF911F910F910895E8EDF0E0808131
:103C30008F7E8083E7EDF0E080818160808381E08A
:103C4000809317040C94CD1DE8EDF0E080818C7F0B
:103C500080831092E20008951092DA001092E10041
:103C600008951F920F920FB60F9211240BB60F9268
:103C70002F933F934F935F936F937F938F939F9374
:103C8000AF93BF93EF93FF938091E10082FF0BC04E
:103C90008091E20082FF07C08091E1008B7F8093DA
:103CA000E1000E94021F8091DA0080FF1FC0809116
:103CB000D80080FF1BC08091DA008E7F8093DA00ED
:103CC0008091D90080FF0DC084E189BD86E189BD66
:103CD00009B400FEFDCF81E0809318040E9477189C
:103CE00005C019BC109218040E9480188091E10050
:103CF00080FF19C08091E20080FF15C08091E20032
:103D00008E7F8093E2008091E20080618093E200E8
:103D10008091D80080628093D80019BC85E08093A0
:103D200018040E947B198091E10084FF30C08091CB
:103D3000E20084FF2CC084E189BD86E189BD09B41D
:103D400000FEFDCF8091D8008F7D8093D8008091B8
:103D5000E1008F7E8093E1008091E2008F7E80936E
:103D6000E2008091E20081608093E200809114047F
:103D7000882311F084E007C08091E30087FD02C032
:103D800081E001C083E0809318040E949019809123
:103D9000E10083FF24C08091E20083FF20C0809176
:103DA000E100877F8093E10082E080931804109205
:103DB00014048091E1008E7F8093E1008091E20005
:103DC0008E7F8093E2008091E20080618093E20028
:103DD00042E060E080E00E94C41A0E948318FF91D4
:103DE000EF91BF91AF919F918F917F916F915F9173
:103DF0004F913F912F910F900BBE0F900FBE0F90E0
:103E00001F9018950895CF93809118048823A1F0EE
:103E1000C091E900CF709091EC00892F817090FDE6
:103E200080E8C82B1092E9008091E80083FD0E9491
:103E3000531CCF70C093E900CF9108959093110364
:103E4000809310030895E0911003F09111033097CF
:103E500021F00190F081E02D099480E00895EF9227
:103E6000FF920F931F93CF93DF93E0911003F09194
:103E700011033097B1F18C010280F381E02D099597
:103E80008091060482FF2DC080FF04C08BE997E07B
:103E90000E94B204E80110E285E9E82E87E0F82EDE
:103EA0008091060480FF0BC088811F928F93FF9240
:103EB000EF920E944B050F900F900F900F901150B2
:103EC00021961111EDCF8091060480FF0AC083E98D
:103ED00097E0DF91CF911F910F91FF90EF900C949D
:103EE000B204DF91CF911F910F91FF90EF90089551
:103EF000E0911003F0911103309721F00480F581D7
:103F0000E02D09940895CF93DF9320910E03309113
:103F10000F032817390709F190930F0380930E03BD
:103F2000E0911003F09111033097B9F0EC01068095
:103F3000F781E02D09958091060482FF0EC080FF75
:103F40000CC0DF93CF9385E897E09F938F930E94F7
:103F50004B050F900F900F900F90DF91CF91089528
:103F6000CF93DF9320910C0330910D03281739076D
:103F700009F190930D0380930C03E0911003F091ED
:103F800011033097B9F0EC010084F185E02D09951B
:103F90008091060482FF0EC080FF0CC0DF93CF9398
:103FA00085E797E09F938F930E944B050F900F90AA
:103FB0000F900F90DF91CF9108950C949E200E9456
:103FC000BD2C0C947A0C8F929F92AF92BF92CF929D
:103FD000DF92EF92FF920F931F93CF93DF9300D066
:103FE00000D01F92CDB7DEB70E94501603E113E058
:103FF000F12C8F2D0E94810C4C01F801A080B18022
:10400000A826B926A114B10439F4F3940E5F1F4F0A
:10401000F8E0FF12EECF39C08091060481FD0E94C6
:10402000B220E12CCC24C394D12CC5018C219D213C
:10403000892B21F1E982FA8221E0C4018C219D21A2
:10404000892B09F420E02B830E94C62C8160782FF5
:104050009D838C8349815A816B818D810E94E820E8
:1040600049815A816B817C818D810E945D2CF80190
:10407000808191818C259D2591838083E394CC0C54
:10408000DD1CF0E1EF12D1CFC0CF8FEF89838A839F
:104090001B820E94C62C8160782F9D838C8349816E
:1040A0005A816B818D810E94E8200E945C2C0E94C5
:1040B000322F0E94231F90911203891759F10E94F9
:1040C000231F809312039091060492FF0EC090FF6D
:1040D0000CC01F928F9386EA97E09F938F930E9464
:1040E0004B050F900F900F900F90809112030F903F
:1040F0000F900F900F900F90DF91CF911F910F9124
:10410000FF90EF90DF90CF90BF90AF909F908F90F7
:104110000C946E2C0F900F900F900F900F90DF91DA
:10412000CF911F910F91FF90EF90DF90CF90BF90B4
:10413000AF909F908F9008950C94B60C0895CF93F4
:10414000C62F0E94810C21E030E002C0220F331FF5
:10415000CA95E2F72823392381E0232B09F480E074
:10416000CF910895EF92FF920F931F93CF93DF9318
:104170008DEB97E00E94B204C0E0D0E080E2E82E30
:1041800081E0F82E01EB17E08C2F0E94810C0E9439
:10419000482CFF92EF929F938F93DF93CF931F93BF
:1041A0000F930E944B0521968DB79EB708960FB6C8
:1041B000F8949EBF0FBE8DBFC830D10529F7DF919F
:1041C000CF911F910F91FF90EF900895089508955A
:1041D000CF93DF93CDB7DEB72B970FB6F894DEBF42
:1041E0000FBECDBF942F4F83252F588769877A87BD
:1041F0008B874A855B85452B31F02F3F31F481E079
:104200009F3F19F403C081E001C080E080FD07C03A
:104210004F81588569857A858B850E945D2CDE01EA
:10422000119686E0FD0111928A95E9F785E0FE017D
:10423000379601900D928A95E1F749815A816B81F9
:104240007C818D819E810E944E282B960FB6F8941A
:10425000DEBF0FBECDBFDF91CF910895882309F453
:10426000BBC09CEF980F913A18F40E942C2B0DC004
:1042700090E2980F983058F4877091E001C0990F40
:104280008A95EAF7892F0E94D12B0C940B2C9BE581
:10429000980F933070F4853A29F0863A31F083E82C
:1042A00090E005C081E890E002C082E890E00C94C4
:1042B000831F98E5980F973108F08EC0883A09F46B
:1042C00045C0893A09F445C08A3A09F445C08B3A99
:1042D00009F445C08C3A09F445C08D3A09F445C04B
:1042E0008E3A09F445C08F3A09F445C0813B09F480
:1042F00045C0803B09F445C0823B09F445C0833B7F
:1043000009F445C0843B09F445C0853B09F445C028
:10431000863B09F445C0873B09F445C0883B09F456
:1043200045C0893B09F445C08A3B09F445C08B3B35
:1043300009F445C08C3B09F445C08D3B09F445C0E8
:104340008E3B09F445C080E090E044C082EE90E0EE
:1043500041C089EE90E03EC08AEE90E03BC085EB24
:1043600090E038C086EB90E035C083EB90E032C03F
:1043700084EB90E02FC087EB90E02CC08CEC90E0B9
:1043800029C08DEC90E026C083E891E023C08AE844
:1043900091E020C082E991E01DC084E991E01AC05B
:1043A00081E292E017C083E292E014C084E292E0DE
:1043B00011C085E292E00EC086E292E00BC087E277
:1043C00092E008C08AE292E005C08FE690E002C069
:1043D00080E790E00C94B01F0895882329F19CEFAA
:1043E000980F913A18F40E947C2B0DC090E2980F20
:1043F000983058F4877091E001C0990F8A95EAF7D8
:10440000892F0E94D72B0C940B2C9BE5980F93308F
:1044100020F480E090E00C94831F885A873120F4C8
:1044200080E090E00C94B01F0895882321F00E9452
:10443000D12B0C940B2C0895882321F00E94D72BAC
:104440000C940B2C08950E94F12B0E94C02B0E940B
:104450000B2C0E94D72F0E94A52E80E090E00E9496
:10446000831F80E090E00C94B01F0E94E12B0C941D
:104470002322CF92DF92EF92FF920F931F93CF935D
:10448000DF9300D000D01F92CDB7DEB76C010E9441
:10449000702C811118C385E0F601DE0111960190A0
:1044A0000D928A95E1F7F601408151812381348193
:1044B0002115310531F05F3F31F481E04F3F19F4B0
:1044C00003C081E001C080E080FDFDC2F601F28002
:1044D000E580E2948FE0E82249835A83FB82722FC1
:1044E0003D832C836F2D8D810E94A82A8C010E9410
:1044F000A72A0E94A129E12FE295EF708E2F90E06C
:10450000FC01EF5BFE4F0C942831812F807F1F70E0
:10451000882311F01295107FFF20B9F0112329F0A4
:10452000812F0E94E42B0E940B2C802F0F900F9064
:104530000F900F900F90DF91CF911F910F91FF90EF
:10454000EF90DF90CF900C942E21802F0E94ED21D0
:10455000112309F4B8C2812F0E94EA2B0F900F900B
:104560000F900F900F90DF91CF911F910F91FF90BF
:10457000EF90DF90CF900C940B2C812F807F1F70D9
:10458000803211F01295107F002319F0013009F1EB
:104590002BC0FF20A9F0EE2059F1F1E0812FEF129E
:1045A00028C00F900F900F900F900F90DF91CF9138
:1045B0001F910F91FF90EF90DF90CF900C94F42B10
:1045C000EE2021F021E0E21609F47DC20E94F72BD3
:1045D0004DC0FF20E9F085E08E1508F474C20E94FA
:1045E000CE2B812329F042C0FF20F1F1E11015C04C
:1045F000812F0F900F900F900F900F90DF91CF9120
:104600001F910F91FF90EF90DF90CF900C941522A7
:1046100094E09E1508F457C229C0F601858180FFF9
:1046200013C08F708583E4CF003F09F489C108F07F
:1046300055C180E4800F803208F459C1FF2009F48D
:10464000EAC1EE2009F49AC1802F0E942E2109337D
:1046500009F0DAC1FFEF21EE84E0F1502040804004
:10466000E1F700C000002FC2E110D7C1812F59C16E
:10467000812F86958695837019F08130B9F023C219
:10468000FF2019F0C801937002C080E090E00F9005
:104690000F900F900F900F90DF91CF911F910F917E
:1046A000FF90EF90DF90CF900C94831FFF2019F0C4
:1046B000C801937002C080E090E00F900F900F90BF
:1046C0000F900F90DF91CF911F910F91FF90EF907E
:1046D000DF90CF900C94B01F802FFF2019F00E9424
:1046E000B82D02C00E94202E0F900F900F900F90B7
:1046F0000F90DF91CF911F910F91FF90EF90DF907E
:10470000CF900C94A52E812F837009F070C0F1100A
:10471000DAC1202F229526952770220F220F602FB5
:104720006F70862F90E0A0E0B0E06C017D01022E5A
:1047300004C0CC0CDD1CEE1CFF1C0A94D2F704FF55
:1047400012C08FE090E0A0E0B0E004C0880F991F95
:10475000AA1FBB1F2A95D2F7BC01CD0160957095A9
:104760008095909503C060E070E0CB01169516959A
:1047700013701230B1F040F56C297D298E299F29E4
:10478000113031F10F900F900F900F900F90DF913B
:10479000CF911F910F91FF90EF90DF90CF900C94ED
:1047A000BC296C297D298E299F290F900F900F908D
:1047B0000F900F90DF91CF911F910F91FF90EF908D
:1047C000DF90CF900C94D6290E94BC29C701B60176
:1047D0000F900F900F900F900F90DF91CF911F913E
:1047E0000F91FF90EF90DF90CF900C94A229FF20C3
:1047F00019F0812F817001C08695882309F463C167
:10480000202F229526952770220F220F602F6F7080
:10481000862F90E0A0E0B0E06C017D01022E04C084
:10482000CC0CDD1CEE1CFF1C0A94D2F704FF12C056
:104830008FE090E0A0E0B0E004C0880F991FAA1FAD
:10484000BB1F2A95D2F7BC01CD016095709580956C
:10485000909503C060E070E0CB011695169513703B
:104860001230B1F040F56C297D298E299F29113035
:1048700031F10F900F900F900F900F90DF91CF912B
:104880001F910F91FF90EF90DF90CF900C94832AAF
:104890006C297D298E299F290F900F900F900F90E2
:1048A0000F90DF91CF911F910F91FF90EF90DF90CC
:1048B000CF900C94952A0E94832AC701B6010F90CD
:1048C0000F900F900F900F90DF91CF911F910F914C
:1048D000FF90EF90DF90CF900C94712A023F09F483
:1048E0005EC008F449C0033F09F46CC0A7CE902F06
:1048F0009071E92E812F8F71FF2051F00E940A2ABA
:10490000802FEE2019F08295807F73CE8F7071CE4C
:104910000E942B2A802FEE2019F08295807F01C003
:104920008F700F900F900F900F900F90DF91CF919D
:104930001F910F91FF90EF90DF90CF900C941C226D
:10494000FF20A9F0E4E0EE1508F4BDC0812F8F71BF
:104950000F900F900F900F900F90DF91CF911F91BC
:104960000F91FF90EF90DF90CF900C94502AF5E0DC
:10497000FE1508F4A8C0EACFFF2099F0812F8F71AF
:104980000F900F900F900F900F90DF91CF911F918C
:104990000F91FF90EF90DF90CF900C940A2AFF20A8
:1049A00069F3812F8F710F900F900F900F900F90E0
:1049B000DF91CF911F910F91FF90EF90DF90CF90FB
:1049C0000C942B2AFF2089F0812F8F710F900F906C
:1049D0000F900F900F90DF91CF911F910F91FF904B
:1049E000EF90DF90CF900C94F5290F900F900F90DF
:1049F0000F900F90DF91CF911F910F91FF90EF904B
:104A0000DF90CF900C94F029033509F423CE0734BE
:104A100009F059C01FCEEE2021F2802F0F900F9089
:104A20000F900F900F90DF91CF911F910F91FF90FA
:104A3000EF90DF90CF900C94ED21412F4F70602FBD
:104A4000C6010E94322D0F900F900F900F900F9083
:104A5000DF91CF911F910F91FF90EF90DF90CF905A
:104A60000C94FC2801112FC0FF2069F10E9435220F
:104A70002FEF80E792E0215080409040E1F700C0A6
:104A800000000F900F900F900F900F90DF91CF913B
:104A90001F910F91FF90EF90DF90CF900C94132D0A
:104AA000412F4F70602FC6010F900F900F900F9005
:104AB0000F90DF91CF911F910F91FF90EF90DF90BA
:104AC000CF900C94352D0F900F900F900F900F906A
:104AD000DF91CF911F910F91FF90EF90DF90CF90DA
:104AE00008951F93CF93DF9300D000D01F92CDB7CE
:104AF000DEB7942F4983252F5A836B837C838D8364
:104B00004C815D81452B31F02F3F31F481E09F3F97
:104B100019F403C081E001C080E0182F117080FDFE
:104B200024C049815A816B817C818D810E94A82A91
:104B3000292F22952F702C3030F42A3048F422503F
:104B4000223068F013C02C3061F02F3051F00EC0CD
:104B5000803C28F0803E50F0815F833038F011E0D7
:104B600005C093FB112710F901C010E0812F0F90B1
:104B70000F900F900F900F90DF91CF911F9108959C
:104B8000CF93DF9300D000D01F92CDB7DEB70F9048
:104B90000F900F900F900F90DF91CF910895CF93CA
:104BA000DF9300D000D000D0CDB7DEB726960FB689
:104BB000F894DEBF0FBECDBFDF91CF9108951F9354
:104BC000CF93DF93C091230316E080912403C8178D
:104BD00099F0D0E01C9FF0011D9FF00D1124EB5DBA
:104BE000FC4F4081518162817381848195810E9453
:104BF000CF252196C770E9CFDF91CF911F910895FE
:104C0000409155035091560360915703709158039A
:104C10008091590390915A030C94CF250F931F93C1
:104C2000CF93DF9380915A0382958F7009F05DC016
:104C300080915703882309F458C080912303109171
:104C400024036091550370915603C0915803D0918D
:104C5000590391E06F3F09F090E0292F06E081179A
:104C600009F443C0209721F07F3F21F030E003C0DA
:104C700031E001C0322F90E030FD34C0089FF001D8
:104C8000099FF00D1124DF01AB5DBC4F11963C91E3
:104C90001197371327C03C91361324C012963C91CC
:104CA000129731111FC013964D915C9114974C1BB4
:104CB0005D0B483C5105B0F480915A038F708061C0
:104CC00080935A03E65DFC4F80818F708061808302
:104CD00085E593E00E943922DF91CF911F910F91DA
:104CE0000C94DF2501968770BACFDF91CF911F9189
:104CF0000F9108959F92AF92BF92CF92DF92EF9261
:104D0000FF920F931F93CF93DF93CDB7DEB76197D9
:104D10000FB6F894DEBF0FBECDBF8C0185E0F80161
:104D2000DE011D9601900D928A95E1F7F801408110
:104D30005181F280C380D4809091550360915603D5
:104D400020915803309159032115310531F06F3FFF
:104D500031F481E09F3F19F403C081E001C080E09D
:104D6000F82FF1709F2E80FD52C185E5A82E83E0BB
:104D7000B82EE0905703F601E21BF30BEE2009F486
:104D8000E8C080915A03E83CF10508F0A4C0282F40
:104D9000207F09F053C0561313C0491311C0EF2CE4
:104DA000F1100EC08F70806180935A030E9400261C
:104DB000C5010E94392280915A03F80185835BC1A5
:104DC000C114D10431F05F3F31F481E04F3F19F459
:104DD00003C081E001C080E080FD03C081E08F2539
:104DE00002C080E090E0F82FF170EF2E80FF1CC031
:104DF000809123032091240336E0821709F418C11F
:104E000090E0389FF001399FF00D1124EB5DFC4FCD
:104E10006181561306C06081461303C06281F61299
:104E200003C001968770E9CFEF2CFF2009F423C15E
:104E300080915A03816080935A0362C0561306C062
:104E4000491304C0F11002C0F801A7C04D875E8766
:104E5000FF867C2DD98AC88A6F2D89890E94712589
:104E6000882399F1FF2089F120915A03822F82959E
:104E70008F7090E0029774F08091550390915603E3
:104E800098878F831986DB86CA862C87CE01079682
:104E90000E94392286E0F801A5E5B3E001900D9269
:104EA0008A95E1F70E940E260E94002611C056172F
:104EB00049F14D875E87FF867C2DD98AC88A6F2D80
:104EC00089890E94712581112CC0C8010E94392254
:104ED000EE24E394D0C0282F207F49F77C2DD98A77
:104EE000C88A6F2D89890E94C02585E593E00E94BC
:104EF000392286E0F50111928A95E9F70E94002691
:104F0000E12CB9C04913D5CFF110D3CFF801858377
:104F1000C8010E94392286E0F50111928A95E9F7CD
:104F2000AAC0FF2091F220915A03822F82958F70A0
:104F300090E002970CF4AECF809155039091560308
:104F40009A8389831B82DD82CC822E83CE010196D7
:104F50009FCFE83CF10508F04BC0EF2CFF2009F48F
:104F6000B4CF561330C049132EC020915A0320FDF0
:104F700021C0822F82958F70482F50E04115510536
:104F8000C9F0F80125834F30510541F08F5F982F0C
:104F90009295907F822F8F70892B8583C8010E9404
:104FA000392286E0F801A5E5B3E001900D928A95DB
:104FB000E1F72AC086E0F801A5E5B3E001900D9283
:104FC0008A95E1F758C04D875E87FF867C2DD98A88
:104FD000C88A6F2D89890E94712581115BCF8091CC
:104FE0005A03816080935A03C8010E94392243C04A
:104FF0007C2DD98AC88A6F2D89890E94C02586E0B8
:10500000F50111928A95E9F70E94002634C0FF202D
:1050100009F45BCF4D875E87FF867C2DD98AC88ACD
:105020006F2D89890E947125882309F44ECF32CFD4
:105030007C2DD98AC88A6F2D89890E94A82A292F98
:1050400022952F70223028F49F7039F0811105C00D
:105050000BC0243028F49F7049F4805E883020F023
:10506000C8010E9439229E2CE92C05C0F8019581C7
:10507000907F99F7F9CF8E2D61960FB6F894DEBF29
:105080000FBECDBFDF91CF911F910F91FF90EF9099
:10509000DF90CF90BF90AF909F9008951F93CF93D4
:1050A000DF93CDB7DEB72C970FB6F894DEBF0FBEF7
:1050B000CDBF4F83588769877A878B879C87CE01BE
:1050C00007960E947A268823D1F09F8188852A85B9
:1050D0003B85232B31F08F3F31F481E09F3F19F462
:1050E00003C081E001C080E080FD47C04F8158854A
:1050F00069857A858B859C850E94CF253EC086E098
:10510000FE013796DE01119601900D928A95E1F726
:10511000FF81E8856A857B856115710531F0EF3F78
:1051200031F481E0FF3F19F403C081E001C080E069
:1051300080FD23C02091240330E0C90101968770CF
:1051400099274091230350E084179507F1F1F983E3
:10515000EA837D836C8396E0929FD001939FB00D8C
:105160001124AB5DBC4FFE01319601900D929A95D2
:10517000E1F7809324030E94DF2516E0809123034A
:1051800090912403891771F1189FC00111248B5D40
:105190009C4F0E947A26882329F1E09123031E9FC9
:1051A000F0011124EB5DFC4F4081518162817381DC
:1051B000848195810E94CF258091230390E0019600
:1051C0008770992780932303D9CF0E9435221092AC
:1051D000240310922303E5E5F3E086E0DF011D924E
:1051E0008A95E9F72C960FB6F894DEBF0FBECDBFB7
:1051F000DF91CF911F910895DF92EF92FF920F936D
:105200001F93CF93DF93FC01892B09F488C0E12C15
:10521000F12CDD24D394EF0121968491853709F494
:1052200060C058F4843708F04EC0843008F068C07D
:105230008130D1F0823071F172C0883709F45BC0DF
:1052400050F4863709F453C0873709F068C08E2DB3
:105250000E94DE2B52C09CE7980F903708F05FC089
:105260008F770E94ED214EC08F010E5F1F4FFE0110
:10527000849190E2980F983050F48770FD2D01C012
:10528000FF0F8A95EAF78F2F0E94E42B15C00E942A
:105290002E2114C08F010E5F1F4FFE01849190E2FA
:1052A000980F983068F48770FD2D01C0FF0F8A9524
:1052B000EAF78F2F0E94EA2B0E940B2CE80122C0F4
:1052C0000E94ED21FBCFCF010296FE01C491CC23B9
:1052D00061F0EFE9FFE03197F1F700C00000C15045
:1052E000F6CFCF010296FE01F490EC010BC00E94B4
:1052F000CE2BE82E07C00E94E12B0E940B2C02C08F
:105300000E942E218F2D882341F0EFE9FFE0319795
:10531000F1F700C000008150F6CFFE017CCFDF9195
:10532000CF911F910F91FF90EF90DF9008956093C0
:10533000DB037093DC038093DD039093DE030C9416
:105340006D2C08950F931F930091DF031091E003DC
:105350002091E1033091E203602B712B822B932B80
:105360006093DF037093E0038093E1039093E20383
:105370001F910F910C946C2C0F931F930091DF03DE
:105380001091E0032091E1033091E2036023712347
:10539000822393236093DF037093E0038093E10300
:1053A0009093E2031F910F910C946C2C0F931F9319
:1053B0000091DF031091E0032091E1033091E203BB
:1053C00060277127822793276093DF037093E003A0
:1053D0008093E1039093E2031F910F910C946C2C46
:1053E00060E070E0CB010C9497290F931F9341E08C
:1053F00050E060E070E08A019B0104C0000F111FC3
:10540000221F331F8A95D2F7C901B8011F910F914E
:105410000C9497290F931F9341E050E060E070E0F7
:1054200004C0440F551F661F771F8A95D2F78091DD
:10543000DB039091DC03A091DD03B091DE038A01D0
:105440009B01082B192B2A2B3B2BC901B8011F915B
:105450000F910C9497290F931F9341E050E060E067
:1054600070E004C0440F551F661F771F8A95D2F75E
:1054700040955095609570958091DB039091DC0389
:10548000A091DD03B091DE038A019B01082319235B
:105490002A233B23C901B8011F910F910C9497292E
:1054A0000F931F9341E050E060E070E004C0440FB0
:1054B000551F661F771F8A95D2F78091DB03909165
:1054C000DC03A091DD03B091DE038A019B01082774
:1054D00019272A273B27C901B8011F910F910C9466
:1054E00097290F931F930091DB031091DC03209108
:1054F000DD033091DE03602B712B822B932B1F91E8
:105500000F910C9497290F931F930091DB03109137
:10551000DC032091DD033091DE03602371238223BD
:1055200093231F910F910C9497290F931F93009130
:10553000DB031091DC032091DD033091DE03602753
:105540007127822793271F910F910C949729089513
:105550008F929F92AF92BF92DF92EF92FF920F9342
:105560001F93CF93DF9300D000D01F92CDB7DEB74B
:105570006B837C838D838A018C819D81892B31F0A3
:105580001F3F31F481E04F3F19F403C081E001C0B7
:1055900080E080FF03C080E090E04DC08B818823D5
:1055A000D1F18090DB039090DC03A090DD03B090FC
:1055B000DE038091DF039091E003A091E103B091BD
:1055C000E203882A992AAA2ABB2A8FE1E82EF12C25
:1055D000D501C4010E2C04C0B695A7959795879563
:1055E0000A94D2F780FD06C081E0E81AF10880F73E
:1055F000D12C07C0DE2CB8018E2D0E948C0C019797
:1056000099F380E1189FF0011124E55AFC4FE00F57
:10561000F11DD08209C080E1189FF0011124E55AE4
:10562000FC4FE00FF11DD08009831A8369817A81D4
:105630008D2D0E948C0C0F900F900F900F900F905B
:10564000DF91CF911F910F91FF90EF90DF90BF906E
:10565000AF909F908F90089590911101992379F1C7
:1056600090911201992359F1982F969596959695B8
:105670009F31A1F0E0911301F0911401E90FF11DA8
:10568000877021E030E0A90102C0440F551F8A95C0
:10569000E2F7CA019181892B8183089590910604D4
:1056A00090FF29C01F928F9380EF97E09F938F9375
:1056B0000E944B050F900F900F900F90089520912E
:1056C000130130911401F90132969FEF40E051919E
:1056D000851789F09F3F19F4511101C0942F4F5F36
:1056E0004E31A9F79F3F39F0F901E90FF11D97FD00
:1056F000FA9582830895089590911101992381F17B
:1057000090911201992361F1982F9695969596950F
:105710009F31A9F0E0911301F0911401E90FF11DFF
:10572000877021E030E0A90102C0440F551F8A951F
:10573000E2F7CA0180959181892381830895909130
:10574000060490FF1CC01F928F9382ED97E09F93F9
:105750008F930E944B050F900F900F900F9008951C
:10576000E0911301F09114019F01225E3F4F92815D
:10577000891301C012823196E217F307C1F7089529
:1057800081E090E0E0911301F0911401E80FF91F1E
:105790001082019680329105A9F708958091050441
:1057A000089590910504892B8093050408958095B0
:1057B000909105048923809305040895809305043E
:1057C000089510920504089590910404892B809304
:1057D000040408958095909104048923809304041F
:1057E00008951092040408958093E303089510929D
:1057F000E30308958091130190911401FC01319607
:105800009C01205E3F4F80E0919191118F5FE217E4
:10581000F307D1F70895E0911301F09114018091FD
:1058200005048083E0911301F0911401908180912F
:105830000404892B80838091E303882361F0E09145
:105840001301F09114019081892B80830E94FA2B1F
:1058500081111092E30380911301909114010C9433
:105860002F1F90937F0180937E0108958295982F3A
:10587000937344E0949F900111248C7C86958695C7
:10588000282B822F8575880F2A7A2695822B0895DA
:10589000CF93DF93D92F0E94362CC82F8D2F0E94D3
:1058A000362C2C2F30E0322F2227A901482BCA0199
:1058B000DF91CF91089508950895CF93DF9300D09D
:1058C00000D01F92CDB7DEB70F900F900F900F90C2
:1058D0000F90DF91CF910895089508950C949C2026
:1058E00080E0089583B7817F8C6083BF83B7816038
:1058F00083BF7894889583B78E7F83BF0895CF93B5
:105900000E94E6200E9450160E94E720C0E08C2FE3
:105910000E94810C892B29F4CF5FC830C1F780E049
:1059200001C081E0CF9108950E948A0C0C94352229
:105930001F920F920FB60F9211248F939F93AF93E4
:10594000BF938091070490910804A0910904B0913D
:105950000A044196A11DB11D809307049093080489
:10596000A0930904B0930A04BF91AF919F918F91C6
:105970000F900FBE0F901F90189582E084BD93E0AA
:1059800095BD9AEF97BD80936E0008952FB7F89458
:105990008091070490910804A0910904B0910A0431
:1059A0002FBF08952FB7F8946091070470910804F1
:1059B0008091090490910A042FBF08959C014FB76C
:1059C000F8948091070490910804A0910904B09183
:1059D0000A044FBF821B930B089578941F920F9275
:1059E0000FB60F9211248F939F93AF93BF93809123
:1059F000070490910804A0910904B0910A0401964B
:105A0000A11DB11D8093070490930804A09309047D
:105A1000B0930A04BF91AF919F918F910F900FBEE9
:105A20000F901F9018950E94B31DF89487E797E791
:105A3000909301088093000887E090EBDC0180934D
:105A4000210490932204A0932304B09324049CE0A7
:105A500088E10FB6F894A895809360000FBE9093EC
:105A60006000FFCF80E090E00895089580910D04DC
:105A700080FF0BC06091180185E0689FB001112480
:105A800075956795759567952BC081FF09C06091E5
:105A9000180185E0689FB00111247595679520C0B5
:105AA00082FF07C06091180185E0689FB001112452
:105AB00017C090910E049923D1F0609117019617A9
:105AC00088F72091180185E0289F90011124929F6A
:105AD000A001939F500D112470E0CA010E9414315F
:105AE0006038710540F46115710519F406C065E070
:105AF00070E0862F08958FE7089581E008958091E2
:105B00000D0480FF08C06091160170E075956795DF
:105B10007595679521C081FF06C06091160170E000
:105B20007595679519C082FF04C06091160170E0F9
:105B300010C090910E04992399F060911501961769
:105B4000A0F780911601899FC001112470E00E9486
:105B500014316038710540F46115710519F406C0FF
:105B600061E070E0862F08958FE7089581E0089541
:105B7000803F21F40E94362D819504C0813F29F495
:105B80000E94362D809311040895823F21F40E94D3
:105B9000362D819504C0833F29F40E94362D8093D1
:105BA00010040895893F19F40E947F2D05C08A3F93
:105BB00031F40E947F2D81958093120408958B3FCC
:105BC00021F40E947F2D819504C08C3F29F40E940E
:105BD0007F2D809313040895843F21F480910F0456
:105BE000816017C0853F21F480910F04826011C04D
:105BF000863F21F480910F0484600BC0873F21F41D
:105C000080910F04886005C0883F31F480910F04B3
:105C1000806180930F0408958D3F21F480910D04DD
:105C200081600BC08E3F21F480910D04826005C01D
:105C30008F3F29F480910D04846080930D040895B2
:105C4000803F39F48091110487FF6CC010921104D9
:105C500069C0813F29F4809111041816BCF362C019
:105C600090911004823F29F497FF5CC010921004B9
:105C700059C0833F19F41916CCF354C0893F41F43D
:105C80008091120418160CF04DC0109212044AC0F4
:105C90008A3F29F48091120487FF44C0F6CF8B3FDE
:105CA00039F48091130487FF3DC0109213043AC069
:105CB0008C3F29F4809113041816BCF333C0843F41
:105CC00021F480910F048E7F17C0853F21F48091CD
:105CD0000F048D7F11C0863F21F480910F048B7FCC
:105CE0000BC0873F21F480910F04877F05C0883F58
:105CF00031F480910F048F7E80930F0413C08D3F89
:105D000021F480910D048E7F0BC08E3F21F4809191
:105D10000D048D7F05C08F3F29F480910D048B7F8A
:105D200080930D048091100481110EC080911104A4
:105D300081110AC080911204811106C08091130460
:105D4000811102C010920E0408958091060483FF11
:105D50007EC085E398E00E94B20480910F041F92F8
:105D60008F9380E398E09F938F930E944B058EE280
:105D700098E00E94B20480911004282F082E000C95
:105D8000330B3F938F938BE298E09F938F930E9406
:105D90004B0589E298E00E94B20480911104282FFB
:105DA000082E000C330B3F938F9386E298E09F936D
:105DB0008F930E944B0584E298E00E94B204809188
:105DC0001204282F082E000C330B3F938F9381E28F
:105DD00098E09F938F930E944B058FE198E00E947B
:105DE000B20480911304282F082E000C330B3F932C
:105DF0008F938CE198E09F938F930E944B0589E1EC
:105E000098E00E94B20480910E041F928F9386E165
:105E100098E09F938F930E944B0584E198E00E9445
:105E2000B20480910D041F928F9381E198E09F93BB
:105E30008F930E944B058EE098E00E94B2048DB7CC
:105E40009EB74C960FB6F8949EBF0FBE8DBF8FE0E5
:105E500094E00E94781F0E94C62C90930C048093BB
:105E60000B0408951F93CF93DF9380910B049091BF
:105E70000C040E94DE2CAC0190910E04992321F0B9
:105E80002091190130E006C020911A018AE0289F74
:105E9000900111244217530708F485C08091100423
:105EA000C0911104D091120410911304811107C004
:105EB000C11175C0D11173C0111171C074C09F3F61
:105EC00019F09F5F90930E04181624F40E94362D4B
:105ED000809310048091100487FF05C00E94362D26
:105EE0008195809310041C1624F40E94362D809313
:105EF00011048091110487FF05C00E94362D819501
:105F00008093110460911004662331F1C091110453
:105F1000CC2311F1062E000C770B880B990B0E94F5
:105F20001B3023E333E343E35FE30E947F300E94AF
:105F3000E32F609310046C2FCC0F770B880B990B19
:105F40000E941B3023E333E343E35FE30E947F308F
:105F50000E94E32F609311041D1624F40E947F2DEC
:105F6000809312048091120487FF05C00E947F2D48
:105F7000819580931204111624F40E947F2D809342
:105F800013048091130487FF05C00E947F2D819523
:105F900080931304DF91CF911F910C94A52E9F3F06
:105FA00009F08FCFA0CFDF91CF911F910895EFE03F
:105FB000F4E085E0DF011D928A95E9F710920E0466
:105FC00010920D0408950E94EA2F6894B1110C9468
:105FD000793008950E945E3088F09F5798F0B92F6D
:105FE0009927B751B0F0E1F0660F771F881F991F0E
:105FF0001AF0BA95C9F714C0B13091F00E94783008
:10600000B1E008950C947830672F782F8827B85F17
:1060100039F0B93FCCF3869577956795B395D9F765
:106020003EF490958095709561957F4F8F4F9F4F6F
:106030000895E89409C097FB3EF49095809570957B
:1060400061957F4F8F4F9F4F9923A9F0F92F96E9C4
:10605000BB279395F695879577956795B795F11139
:10606000F8CFFAF4BB0F11F460FF1BC06F5F7F4FD6
:106070008F4F9F4F16C0882311F096E911C07723E8
:1060800021F09EE8872F762F05C0662371F096E8F1
:10609000862F70E060E02AF09A95660F771F881FC0
:1060A000DAF7880F9695879597F9089557FD9058D8
:1060B000440F551F59F05F3F71F04795880F97FBCC
:1060C000991F61F09F3F79F0879508951216130686
:1060D0001406551FF2CF4695F1DF08C016161706B5
:1060E0001806991FF1CF86957105610508940895EA
:1060F000E894BB2766277727CB0197F908950E947C
:1061000092300C9403310E94F53038F00E94FC303C
:1061100020F0952311F00C94EC300C94F230112403
:106120000C9479300E94563070F3959FC1F3950F0F
:1061300050E0551F629FF001729FBB27F00DB11D0B
:10614000639FAA27F00DB11DAA1F649F6627B00D9B
:10615000A11D661F829F2227B00DA11D621F739F84
:10616000B00DA11D621F839FA00D611D221F749F92
:106170003327A00D611D231F849F600D211D822FD9
:10618000762F6A2F11249F5750409AF0F1F0882300
:106190004AF0EE0FFF1FBB1F661F771F881F91502D
:1061A0005040A9F79E3F510580F00C94EC300C94C0
:1061B00079305F3FE4F3983ED4F386957795679501
:1061C000B795F795E7959F5FC1F7FE2B880F911D57
:1061D0009695879597F9089597F99F6780E870E0FD
:1061E00060E008959FEF80EC089500240A9416164D
:1061F000170618060906089500240A9412161306B5
:10620000140605060895092E0394000C11F4882342
:1062100052F0BB0F40F4BF2B11F460FF04C06F5F5E
:106220007F4F8F4F9F4F089597FB072E16F40094D2
:1062300007D077FD09D00E94313107FC05D03EF42C
:10624000909581959F4F0895709561957F4F089522
:10625000EE0FFF1F0024001C0BBE0790F691E02DEF
:106260000994AA1BBB1B51E107C0AA1FBB1FA6179D
:10627000B70710F0A61BB70B881F991F5A95A9F7EF
:0E62800080959095BC01CD010895F894FFCF54
:10628E0005EA010000FF7C161E17EF16B3167F16E7
:10629E00010101E4032808140A321E5F5A31353019
:1062AE00005F3F3F3F3F005F415438340041540090
:1062BE005854005445524D494E414C004E4F4E4598
:1062CE00004D4F55534500494E54454C4C49004CDA
:1062DE004F474954454348004558504C4F5245523C
:1062EE000044454641554C5400397F223C07BD06BB
:0E62FE009B06470660067906001000080004A3
:106800008800EA44E944E244040005000600070069
:10681000080009000A000B000C000D000E000F001C
:1068200010001100120013001400150016001700CC
:10683000180019001A001B001C001D001E001F007C
:10684000200021002200230024002500260027002C
:10685000280029002A002B002C002D002E002F00DC
:10686000300031003200330034003500360037008C
:10687000380039003A003B003C003D003E003F003C
:1068800040004100420043004400450046004700EC
:10689000480049004A004B004C004D004E004F009C
:1068A000500051005200530054005500560057004C
:1068B000580059005A005B005C005D005E005F00FC
:1068C0006000610062006300640065A185006700EC
:1068D000680069006A006B006C006D006E006F005C
:1068E0007000710072007300890087008A008B00BD
:1068F000E000E100E200E300E400E500E600E7007C
:106900000100010001000100EA4401000100E2442D
:106910000100010001000100460001004A004B0097
:10692000010001004700480001000100E9440100A6
:106930000100010001000100010001003A003B00DC
:106940003C003D003E003F0040004100420043004B
:10695000010035004C0039000100440045005200A0
:1069600049000100010050004F0029004D004E0079
:1069700051000100010001000100010001000100BF
:1069800001000100010001000100010001000100FF
:1069900001000100010001000100010001004D00A3
:1069A0004A004E004B0001000100010001000100FF
:1069B00001000100010001000100010001000100CF
:1069C00001000100010001000100010001000100BF
:1069D00001000100010001000100010001000100AF
:1069E0000100010001000100490001000100010057
:1069F000010001000100010001000100010001008F
:00000001FF
